:020000020000FC
:100000001FC0000000000000000075C0CEC000004E
:10001000D0C0E4C000000000000000000D0A626BC8
:100020002473626C2D666C6F682474303570776D44
:100030005F3423335F326B687A5F32306B5F0D0A57
:1000400004E00EBF0FE50DBF03E008BB00E007BBF7
:100050000CE205BB0EE304BB05E102BB0AE101BBF8
:1000600002E003BF02E80EBD772788279927BB2748
:10007000A0E600270D93A338E8F39FD202E0C02E3C
:1000800010B31570153069F0143041F0113019F0CB
:1000900001E011E008C00CE01AE005C008E114E13D
:1000A00002C002E318E200937D0010937E00909856
:1000B000919816D115D1E8D007D1E9D005D1EAD071
:1000C00003D10DE7402E01EF302E00E0D02E882422
:1000D00005E308BF09BF04D1E0D0DFD0DED07894BB
:1000E0008ED20EE100937F0066D1B2C2AA9902C0FF
:1000F000AA9A01C0AA982FB646B557B5882091F0A4
:10010000AAF46EB56F7B6EBD882471FD3FC073FF8E
:100110003DC046195709A42EB52E7260777F42E084
:10012000C42E34C071FD32C0839430C0682D61305C
:1001300021F4642E752E839429C04F935F93461942
:1001400057097F906F90403961E05607E8F04835D5
:1001500062E05607C8F472FD05C040937B005093DF
:100160007C0074604EB540644EBD40E8842EB0996A
:1001700002C078600BC04427A42EB42E726042E007
:10018000C42E4EB54F7B4EBD8824777F2FBE189569
:100190000000000000000000000000000000AA991C
:1001A00002C0AA9A01C0AA98F1CF2FB67E7F2FBEB7
:1001B00018952FB67068EE2009F0EA94CC2059F417
:1001C000B09B04C04427A42EB42E06C0A090770094
:1001D000B090780001C0CA942FBE18952FB676FD56
:1001E00031C0906145999F7E432D552D541738F4A9
:1001F0004A9469F450917D00452E4A9507C039F024
:100200004A9429F450917E00452E4395342E706413
:1002100075FF03C081FF939807C074FF03C081FF7F
:10022000A99802C081FFAC98432D425A3AF44A5F24
:10023000433040F047704A95F1F704C0409545952A
:1002400042BF1EC075FF03C080FF939A07C074FFB2
:1002500003C080FFA99A02C080FFAC9A432D4F9340
:10026000459542BF4F917F7B4D3918F482608E7F58
:1002700007C0413F18F08D7F816002C08D7F8E7F67
:1002800093FD81602FBE189538EC10E509C034EB62
:1002900014E606C030EA18E703C034E618EC00C0E4
:1002A000002702BFAD98A99A02B70032E9F7AD9ACC
:1002B000A99828E0002702BF02B70317E9F72A959B
:1002C000C9F71A9569F708951FE028E0002702BFD3
:1002D00002B70F3FE9F72A95C9F71A95B1F70895C4
:1002E00010E828E0002702BF02B70F3FE9F72A9580
:1002F000C9F71A95B1F708958F7E71FF01C0797F14
:100300000A2D1B2D2091770030917800201731079E
:1003100020F40091770010917800169507951695B6
:1003200007952EE0002371F010917900109F212D88
:1003300010917A00109F200D243608F024E62F300B
:1003400008F42FE0F22F08958F7B20916C0010911C
:100350006B0000916A00011B00936A0000916B0022
:10036000020B00936B0000916C00004000936C0046
:1003700020916900109168000091670026951795FB
:100380000795269517950795209369002093680097
:100390002093670020916A00200F20936A0020912B
:1003A0006B00211F20936B0000E020916C00201F48
:1003B00020936C000895C0E8DBEBC0937100D093EC
:1003C00072002FEF3FE120936D0030936E00209379
:1003D0006F0030937000E1E0E09366003FEF3093F0
:1003E00065002FEF209364000895F89400000CB589
:1003F0001DB500936000109361000C0F1D1F1BBD05
:100400000ABD716078940091640010916500E091DC
:1004100066000093730010937400EE2329F03FEF01
:100420003093730030937400E69517950795E69521
:10043000179507952091640030916500E091660062
:10044000201B310BE0400091600010916100C091D1
:100450006200D091630000936200109363000C1B54
:100460001D0B0093750010937600200F311F10E0D4
:10047000E11FEE2351F4332341F4213E30F431E007
:100480002CE4FF2011F40FEFF02E20936400309342
:100490006500E0936600E23008F09DDF00916700A0
:1004A000020F0093670000916800031F009368002B
:1004B000009169000E1F00936900E6953795279516
:1004C000E69537952795E69537952795E6953795DF
:1004D000279520936D0030936E0020936F0030932A
:1004E00070000895C0916D00D0916E007EDF089578
:1004F00070FDFECFD0917400C0917300F89400009D
:100500000CB51DB50C0F1D1F1BBD0ABD7160789485
:100510000895C0916F00D0917000F89400000CB560
:100520001DB50C0F1D1F1BBD0ABD7160789484FDA5
:10053000E3DE85FD16D086FD07DF70FDFECF089552
:10054000C0917100D091720050DF009160000F7077
:10055000D01BDC3808F4DBEBD093720040D03FD0E6
:1005600008958F7D0F2F0D1908F40EE0109166008D
:10057000112321F410916500103438F091609260DD
:1005800019E1011760F0012F0AC0103238F09E7F88
:10059000926012E3011718F0012F01C09C7F95FFB4
:1005A00009C02EE1021710F40EE104C028E2021780
:1005B00008F0022F0095502E0895FEE001EF302E36
:1005C000502E0CE205BB05E102BB0DE7402E816019
:1005D000977F9062089504E00A95F1F7089576FDFB
:1005E000FECF76FFFECF0895797F71FFFECF797F32
:1005F00071FFFECF00917B0010917C000895F4DF25
:10060000202F312FF1DF021B130B10F410950095F2
:100610001123A9F7007F002391F7209377003093EF
:100620007800369527953695279500E014E6332710
:10063000EE273395332309F4E395021B3F933327C9
:10064000130B3F91B0F730937900E0937A0008954F
:10065000B4DF52DEFF30E8F30EE10095502E3798FC
:1006600000B7086000BF332703E008BB05E102BB09
:100670000BE10A95F1F73AD143D19B7F00E000935B
:10068000800008E2E02E97DE5BDF94FF10C070FD73
:1006900002C0946013C0A3DF94FDF9CF00E0009383
:1006A0008000E6D0EFD003D127DE4ADF31C070FDF5
:1006B00002C0946003C093DF94FFF9CFD9D040DF2C
:1006C00094FD08C070FD02C094600BC088DF94FFE9
:1006D000F9CF07C070FD02C0946003C080DF94FDB5
:1006E000F9CFD0D009DE2CDF94FF08C070FD02C026
:1006F00094600BC074DF94FDF9CF07C070FD02C099
:10070000946003C06CDF94FFF9CFD1D02ADF18DFEB
:1007100094FD08C070FD02C094600BC060DF94FFC0
:10072000F9CF07C070FD02C0946003C058DF94FD8C
:10073000F9CFC7D005DF94FF08C070FD02C09460F8
:100740000BC04DDF94FDF9CF07C070FD02C094606F
:1007500003C045DF94FFF9CFC9D0F2DE94FD08C095
:1007600070FD02C094600BC03ADF94FFF9CF07C060
:1007700070FD02C0946003C032DF94FDF9CFC0D099
:10078000032D013F09F464CFEE2021F461CFEE2068
:1007900009F45ECF00916600002321F4009165000A
:1007A000003250F00091800092FD002703950093E5
:1007B00080009B7F0C3338F00FEFF02E93DE9ADE33
:1007C0009F7D7B7F02C0BCDE60CF4AD070FF2EC011
:1007D00080649FDE4DD086DE8BDE3AD070FF26C06F
:1007E000806197DE4FD07EDE83DE3AD070FF1EC080
:1007F00080628FDE5CD076DE7BDE2AD070FF16C092
:1008000088DE5FD06FDE74DE2BD070FF0FC081DE1C
:100810006DD068DE6DDE1CD070FF08C07ADE70D04F
:1008200061DE66DE00916600002319F09062977F1A
:100830000FCF977FFF2041F0FA9429F00F2D013060
:1008400011F0023009F49860C0CFF894B6DEF8CB0E
:1008500070FF0895459BFCCFBEDE459BF9CF089500
:1008600070FF08954599FCCFB6DE4599F9CF0895FC
:10087000AD9A80FFAB9807E007B9379800B70860DA
:1008800000BF089504E309BF00007F7E7F7D81FDE6
:1008900002C076FD03C0939880FFAC9A05E309BFC0
:1008A00006E007B9379800B7086000BF0895AB9A13
:1008B00080FF949800E007B9379800B7086000BF40
:1008C000089504E309BF000070617F7D81FD02C0CF
:1008D00076FD03C0AC9880FFA99A05E309BF07E045
:1008E00007B9379800B7086000BF0895949A80FF51
:1008F000AD9806E007B9379800B7086000BF0895C3
:1009000004E309BF00007F7E706281FD02C076FDB6
:1009100003C0A99880FF939A05E309BF00E007B9D7
:0A092000379800B7086000BF089583
:00000001FF
